BL51 BANKED LINKER/LOCATER V6.05                                                        07/31/2012  00:51:22  PAGE 1


BL51 BANKED LINKER/LOCATER V6.05, INVOKED BY:
D:\PROGRAM FILES\KEIL_51\C51\BIN\BL51.EXE task.obj, main.obj, zimo.obj, IR_Receive.obj, DS1302.obj, ShowTime.obj, uart.o
>> bj, eeprom58.obj TO xuanzhuan RAMSIZE (256)


MEMORY MODEL: LARGE


INPUT MODULES INCLUDED:
  task.obj (TASK)
  main.obj (MAIN)
  zimo.obj (ZIMO)
  IR_Receive.obj (IR_RECEIVE)
  DS1302.obj (DS1302)
  ShowTime.obj (SHOWTIME)
  uart.obj (UART)
  eeprom58.obj (EEPROM58)
  D:\PROGRAM FILES\KEIL_51\C51\LIB\C51L.LIB (?C_STARTUP)
  D:\PROGRAM FILES\KEIL_51\C51\LIB\C51L.LIB (?C?CLDPTR)
  D:\PROGRAM FILES\KEIL_51\C51\LIB\C51L.LIB (?C?UIDIV)
  D:\PROGRAM FILES\KEIL_51\C51\LIB\C51L.LIB (?C?IILDX)
  D:\PROGRAM FILES\KEIL_51\C51\LIB\C51L.LIB (?C?OFFXADD)
  D:\PROGRAM FILES\KEIL_51\C51\LIB\C51L.LIB (?C?CCASE)
  D:\PROGRAM FILES\KEIL_51\C51\LIB\C51L.LIB (?C_INIT)


LINK MAP OF MODULE:  xuanzhuan (TASK)


            TYPE    BASE      LENGTH    RELOCATION   SEGMENT NAME
            -----------------------------------------------------

            * * * * * * *   D A T A   M E M O R Y   * * * * * * *
            REG     0000H     0008H     ABSOLUTE     "REG BANK 0"
            DATA    0008H     0008H     UNIT         ?DT?TASK
            REG     0010H     0008H     ABSOLUTE     "REG BANK 2"
                    0018H     0008H                  *** GAP ***
            BIT     0020H.0   0000H.2   UNIT         ?BI?IR_RECEIVE
            BIT     0020H.2   0000H.1   UNIT         ?BI?TASK
            BIT     0020H.3   0000H.1   UNIT         ?BI?MAIN
            BIT     0020H.4   0000H.1   UNIT         ?BI?SHOWTIME
            BIT     0020H.5   0000H.1   UNIT         ?BI?UART
                    0020H.6   0000H.2                *** GAP ***
            IDATA   0021H     0001H     UNIT         ?STACK

            * * * * * * *  X D A T A   M E M O R Y  * * * * * * *
            XDATA   0000H     00E1H     UNIT         ?XD?UART
            XDATA   00E1H     0018H     UNIT         ?XD?IR_RECEIVE
            XDATA   00F9H     000EH     UNIT         ?XD?DS1302
            XDATA   0107H     000DH     UNIT         ?XD?TASK
            XDATA   0114H     0006H     UNIT         _XDATA_GROUP_
            XDATA   011AH     0002H     UNIT         ?XD?EEPROM58
            XDATA   011CH     0001H     UNIT         ?XD?SHOWTIME

            * * * * * * *   C O D E   M E M O R Y   * * * * * * *
            CODE    0000H     0003H     ABSOLUTE     
            CODE    0003H     0003H     ABSOLUTE     
            CODE    0006H     000DH     UNIT         ?PR?_W1302?DS1302
BL51 BANKED LINKER/LOCATER V6.05                                                      07/31/2012  00:51:22  PAGE 2


            CODE    0013H     0003H     ABSOLUTE     
                    0016H     0005H                  *** GAP ***
            CODE    001BH     0003H     ABSOLUTE     
                    001EH     0005H                  *** GAP ***
            CODE    0023H     0003H     ABSOLUTE     
            CODE    0026H     0013H     UNIT         ?PR?TIM1_ISR?IR_RECEIVE
                    0039H     0002H                  *** GAP ***
            CODE    003BH     0003H     ABSOLUTE     
            CODE    003EH     07A0H     UNIT         ?CO?ZIMO
            CODE    07DEH     06CEH     UNIT         ?PR?DISPLAY?SHOWTIME
            CODE    0EACH     026CH     UNIT         ?PR?OS_ALLRUN?TASK
            CODE    1118H     0193H     UNIT         ?PR?MAIN_RS_INT?UART
            CODE    12ABH     0185H     UNIT         ?PR?PCA?TASK
            CODE    1430H     00E1H     UNIT         ?PR?_SET?DS1302
            CODE    1511H     00B6H     UNIT         ?C?LIB_CODE
            CODE    15C7H     008CH     UNIT         ?C_C51STARTUP
            CODE    1653H     008BH     UNIT         ?PR?EX1_ISR?IR_RECEIVE
            CODE    16DEH     004FH     UNIT         ?C_INITSEG
            CODE    172DH     0048H     UNIT         ?PR?IRCORDPRO?IR_RECEIVE
            CODE    1775H     0045H     UNIT         ?PR?DU1302?DS1302
            CODE    17BAH     0043H     UNIT         ?PR?INIT?MAIN
            CODE    17FDH     003EH     UNIT         ?PR?START?TASK
            CODE    183BH     0034H     UNIT         ?PR?_SET1302?DS1302
            CODE    186FH     0028H     UNIT         ?PR?_BYTE_READ?EEPROM58
            CODE    1897H     0026H     UNIT         ?PR?_BYTE_PROGRAM?EEPROM58
            CODE    18BDH     0022H     UNIT         ?PR?_SECTOR_ERASE?EEPROM58
            CODE    18DFH     001DH     UNIT         ?PR?_DELAY?TASK
            CODE    18FCH     0016H     UNIT         ?PR?INT0?TASK
            CODE    1912H     0016H     UNIT         ?PR?_RTINPUTBYTE?DS1302
            CODE    1928H     0011H     UNIT         ?PR?_R1302?DS1302
            CODE    1939H     0010H     UNIT         ?PR?RTOUTPUTBYTE?DS1302
            CODE    1949H     000CH     UNIT         ?PR?_SEND_DATA?UART
            CODE    1955H     000CH     UNIT         ?PR?IAP_DISABLE?EEPROM58
            CODE    1961H     000BH     UNIT         ?PR?MAIN?MAIN



OVERLAY MAP OF MODULE:   xuanzhuan (TASK)


SEGMENT                              XDATA_GROUP
  +--> CALLED SEGMENT              START    LENGTH
--------------------------------------------------
?PR?MAIN_RS_INT?UART               0114H    0001H
  +--> ?PR?_SECTOR_ERASE?EEPROM58
  +--> ?PR?_BYTE_PROGRAM?EEPROM58
  +--> ?PR?_SEND_DATA?UART

?PR?_SECTOR_ERASE?EEPROM58         -----    -----
  +--> ?PR?IAP_DISABLE?EEPROM58

?PR?_BYTE_PROGRAM?EEPROM58         -----    -----
  +--> ?PR?IAP_DISABLE?EEPROM58

*** NEW ROOT ***************************************************

?C_C51STARTUP                      -----    -----
BL51 BANKED LINKER/LOCATER V6.05                                                      07/31/2012  00:51:22  PAGE 3


  +--> ?PR?MAIN?MAIN
  +--> ?C_INITSEG

?PR?MAIN?MAIN                      -----    -----
  +--> ?PR?INIT?MAIN
  +--> ?PR?START?TASK
  +--> ?PR?OS_ALLRUN?TASK

?PR?START?TASK                     -----    -----
  +--> ?PR?_BYTE_READ?EEPROM58
  +--> ?PR?_SEND_DATA?UART

?PR?_BYTE_READ?EEPROM58            -----    -----
  +--> ?PR?IAP_DISABLE?EEPROM58

?PR?OS_ALLRUN?TASK                 -----    -----
  +--> ?PR?IRCORDPRO?IR_RECEIVE
  +--> ?PR?_SET?DS1302
  +--> ?PR?_SET1302?DS1302
  +--> ?PR?_W1302?DS1302
  +--> ?PR?_BYTE_READ?EEPROM58
  +--> ?PR?_DELAY?TASK
  +--> ?PR?DU1302?DS1302
  +--> ?PR?DISPLAY?SHOWTIME
  +--> ?CO?ZIMO

?PR?_SET?DS1302                    0115H    0005H
  +--> ?PR?_R1302?DS1302
  +--> ?PR?_W1302?DS1302

?PR?_R1302?DS1302                  -----    -----
  +--> ?PR?_RTINPUTBYTE?DS1302
  +--> ?PR?RTOUTPUTBYTE?DS1302

?PR?_W1302?DS1302                  -----    -----
  +--> ?PR?_RTINPUTBYTE?DS1302

?PR?_SET1302?DS1302                -----    -----
  +--> ?PR?_W1302?DS1302

?PR?DU1302?DS1302                  -----    -----
  +--> ?PR?_R1302?DS1302

?PR?DISPLAY?SHOWTIME               0115H    0001H
  +--> ?CO?ZIMO
  +--> ?PR?_DELAY?TASK



SYMBOL TABLE OF MODULE:  xuanzhuan (TASK)

  VALUE           TYPE          NAME
  ----------------------------------

  -------         MODULE        TASK
  C:0000H         SYMBOL        _ICE_DUMMY_
  D:0080H         PUBLIC        P0
BL51 BANKED LINKER/LOCATER V6.05                                                      07/31/2012  00:51:22  PAGE 4


  D:0090H         PUBLIC        P1
  D:00A0H         PUBLIC        P2
  D:00B0H         PUBLIC        P3
  D:00C0H         PUBLIC        P4
  D:00C8H         PUBLIC        P5
  D:00F9H         PUBLIC        CH
  D:00A8H         PUBLIC        IE
  D:00E9H         PUBLIC        CL
  X:0107H         PUBLIC        DelayTimeCount
  X:0108H         PUBLIC        uitime
  X:010AH         PUBLIC        BuffCount
  C:18DFH         PUBLIC        _delay
  C:0EACH         PUBLIC        OS_ALLRun
  B:00D8H.6       PUBLIC        CR
  D:00DAH         PUBLIC        CCAPM0
  D:00DBH         PUBLIC        CCAPM1
  D:00B8H         PUBLIC        IP
  D:00D8H         PUBLIC        CCON
  D:0008H         PUBLIC        uiBaseAddress
  C:17FDH         PUBLIC        start
  D:000AH         PUBLIC        uiicountTwo
  D:0098H         PUBLIC        SCON
  D:0088H         PUBLIC        TCON
  D:000CH         PUBLIC        ucNumRows
  B:00B0H.0       PUBLIC        Led1
  B:00B0H.1       PUBLIC        Led2
  B:00B0H.4       PUBLIC        Led3
  B:0020H.2       PUBLIC        BIT_timeout
  X:010BH         PUBLIC        S
  C:12ABH         PUBLIC        PCA
  B:0088H.4       PUBLIC        TR0
  X:010DH         PUBLIC        ucPCA0_TimeCount
  X:010EH         PUBLIC        ucMode
  D:000EH         PUBLIC        uiFontNumber
  X:010FH         PUBLIC        Delay
  X:0110H         PUBLIC        uiCountFontNumber
  X:0112H         PUBLIC        uiicount
  D:00D0H         PUBLIC        PSW
  C:18FCH         PUBLIC        int0
  B:00D8H.0       PUBLIC        CCF0
  B:00D8H.1       PUBLIC        CCF1
  -------         PROC          _DELAY
  D:0007H         SYMBOL        n
  -------         DO            
  D:0005H         SYMBOL        a
  D:0006H         SYMBOL        b
  -------         ENDDO         
  C:18DFH         LINE#         37
  C:18DFH         LINE#         38
  C:18DFH         LINE#         40
  C:18E5H         LINE#         41
  C:18E5H         LINE#         42
  C:18E7H         LINE#         43
  C:18F8H         LINE#         44
  C:18FBH         LINE#         45
  -------         ENDPROC       _DELAY
  -------         PROC          PCA
BL51 BANKED LINKER/LOCATER V6.05                                                      07/31/2012  00:51:22  PAGE 5


  C:12ABH         LINE#         48
  C:12C6H         LINE#         50
  C:12C9H         LINE#         51
  C:12C9H         LINE#         52
  C:12CBH         LINE#         53
  C:12CEH         LINE#         54
  C:12D1H         LINE#         55
  C:12D7H         LINE#         56
  C:12DDH         LINE#         57
  C:12DDH         LINE#         58
  C:12DFH         LINE#         59
  C:12E1H         LINE#         60
  C:12E1H         LINE#         61
  C:12E1H         LINE#         63
  C:12E7H         LINE#         64
  C:12E7H         LINE#         65
  C:12E9H         LINE#         66
  C:12ECH         LINE#         67
  C:12EFH         LINE#         68
  C:12FDH         LINE#         69
  C:1334H         LINE#         70
  C:1334H         LINE#         71
  C:1334H         LINE#         73
  C:1334H         LINE#         75
  C:1334H         LINE#         77
  C:1334H         LINE#         79
  C:1334H         LINE#         81
  C:1334H         LINE#         83
  C:1334H         LINE#         85
  C:1334H         LINE#         87
  C:1334H         LINE#         89
  C:1334H         LINE#         91
  C:1334H         LINE#         93
  C:1334H         LINE#         95
  C:1337H         LINE#         96
  C:1341H         LINE#         97
  C:1341H         LINE#         101
  C:1341H         LINE#         104
  C:136FH         LINE#         105
  C:136FH         LINE#         106
  C:1372H         LINE#         107
  C:1374H         LINE#         108
  C:1376H         LINE#         109
  C:1378H         LINE#         110
  C:137AH         LINE#         111
  C:1384H         LINE#         112
  C:1384H         LINE#         114
  C:13B2H         LINE#         115
  C:13B2H         LINE#         116
  C:13B5H         LINE#         117
  C:13B7H         LINE#         118
  C:13B9H         LINE#         119
  C:13BBH         LINE#         120
  C:13BDH         LINE#         121
  C:13C7H         LINE#         122
  C:13C7H         LINE#         125
  C:13F5H         LINE#         126
BL51 BANKED LINKER/LOCATER V6.05                                                      07/31/2012  00:51:22  PAGE 6


  C:13F5H         LINE#         127
  C:13F8H         LINE#         128
  C:13FBH         LINE#         129
  C:13FDH         LINE#         130
  C:13FFH         LINE#         131
  C:1401H         LINE#         132
  C:140BH         LINE#         133
  C:140BH         LINE#         135
  C:140EH         LINE#         136
  C:1411H         LINE#         137
  C:1413H         LINE#         138
  C:1415H         LINE#         139
  C:1417H         LINE#         141
  C:1417H         LINE#         142
  -------         ENDPROC       PCA
  -------         PROC          INT0
  C:18FCH         LINE#         146
  C:1902H         LINE#         148
  C:1909H         LINE#         149
  C:190BH         LINE#         150
  -------         ENDPROC       INT0
  -------         PROC          START
  C:17FDH         LINE#         152
  C:17FDH         LINE#         153
  C:17FDH         LINE#         154
  C:1800H         LINE#         155
  C:1803H         LINE#         156
  C:1806H         LINE#         157
  C:1809H         LINE#         158
  C:180CH         LINE#         159
  C:180FH         LINE#         160
  C:1832H         LINE#         161
  C:1836H         LINE#         162
  -------         ENDPROC       START
  -------         PROC          OS_ALLRUN
  C:0EACH         LINE#         166
  C:0EACH         LINE#         167
  C:0EACH         LINE#         169
  C:0EB2H         LINE#         170
  C:0EB2H         LINE#         171
  C:0EB4H         LINE#         172
  C:0EBAH         LINE#         173
  C:0EBAH         LINE#         174
  C:0EBDH         LINE#         175
  C:0EBFH         LINE#         176
  C:0EE8H         LINE#         177
  C:0EE8H         LINE#         178
  C:0EE8H         LINE#         179
  C:0EEEH         LINE#         180
  C:0EF1H         LINE#         182
  C:0EF1H         LINE#         183
  C:0EFDH         LINE#         184
  C:0F00H         LINE#         185
  C:0F02H         LINE#         187
  C:0F02H         LINE#         188
  C:0F07H         LINE#         189
  C:0F07H         LINE#         190
BL51 BANKED LINKER/LOCATER V6.05                                                      07/31/2012  00:51:22  PAGE 7


  C:0F07H         LINE#         191
  C:0F09H         LINE#         193
  C:0F09H         LINE#         194
  C:0F0BH         LINE#         195
  C:0F0DH         LINE#         196
  C:0F13H         LINE#         197
  C:0F15H         LINE#         199
  C:0F15H         LINE#         200
  C:0F1BH         LINE#         201
  C:0F1DH         LINE#         202
  C:0F1FH         LINE#         203
  C:0F22H         LINE#         204
  C:0F25H         LINE#         205
  C:0F27H         LINE#         206
  C:0F27H         LINE#         207
  C:0F2DH         LINE#         208
  C:0F2FH         LINE#         209
  C:0F31H         LINE#         210
  C:0F33H         LINE#         212
  C:0F33H         LINE#         213
  C:0F3AH         LINE#         214
  C:0F3CH         LINE#         216
  C:0F3CH         LINE#         217
  C:0F46H         LINE#         218
  C:0F48H         LINE#         220
  C:0F48H         LINE#         221
  C:0F4EH         LINE#         222
  C:0F51H         LINE#         223
  C:0F54H         LINE#         224
  C:0F56H         LINE#         225
  C:0F5CH         LINE#         226
  C:0F5CH         LINE#         227
  C:0F5EH         LINE#         228
  C:0F60H         LINE#         229
  C:0F62H         LINE#         230
  C:0F62H         LINE#         231
  C:0F64H         LINE#         232
  C:0F64H         LINE#         233
  C:0F6DH         LINE#         234
  C:0F74H         LINE#         235
  C:0F7BH         LINE#         236
  C:0F7BH         LINE#         238
  C:0F7BH         LINE#         239
  C:0F7BH         LINE#         240
  C:0F7BH         LINE#         243
  C:0F99H         LINE#         244
  C:0F99H         LINE#         245
  C:0F99H         LINE#         247
  C:0FB5H         LINE#         248
  C:0FB5H         LINE#         250
  C:0FBCH         LINE#         252
  C:0FBCH         LINE#         253
  C:0FE8H         LINE#         254
  C:0FE8H         LINE#         257
  C:0FFBH         LINE#         258
  C:1015H         LINE#         259
  C:1033H         LINE#         260
BL51 BANKED LINKER/LOCATER V6.05                                                      07/31/2012  00:51:22  PAGE 8


  C:1038H         LINE#         261
  C:1041H         LINE#         262
  C:1047H         LINE#         263
  C:1047H         LINE#         265
  C:1047H         LINE#         266
  C:1047H         LINE#         267
  C:1058H         LINE#         268
  C:1058H         LINE#         269
  C:1058H         LINE#         270
  C:105BH         LINE#         272
  C:105EH         LINE#         273
  C:105EH         LINE#         275
  C:105EH         LINE#         277
  C:1061H         LINE#         278
  C:1073H         LINE#         279
  C:1085H         LINE#         280
  C:1097H         LINE#         282
  C:1098H         LINE#         283
  C:1098H         LINE#         284
  C:10A6H         LINE#         285
  C:10B5H         LINE#         286
  C:10B5H         LINE#         287
  C:10B9H         LINE#         288
  C:10B9H         LINE#         289
  C:10DAH         LINE#         290
  C:10DAH         LINE#         291
  C:10F1H         LINE#         292
  C:10FFH         LINE#         293
  C:1104H         LINE#         294
  C:1107H         LINE#         295
  C:110AH         LINE#         297
  C:110DH         LINE#         298
  C:110DH         LINE#         300
  C:110DH         LINE#         301
  C:110DH         LINE#         302
  C:1117H         LINE#         303
  C:1117H         LINE#         304
  C:1117H         LINE#         305
  C:1117H         LINE#         306
  C:1117H         LINE#         308
  C:1117H         LINE#         309
  -------         ENDPROC       OS_ALLRUN
  -------         ENDMOD        TASK

  -------         MODULE        MAIN
  C:0000H         SYMBOL        _ICE_DUMMY_
  B:00A8H.7       PUBLIC        EA
  D:00F9H         PUBLIC        CH
  D:00A8H         PUBLIC        IE
  D:00E9H         PUBLIC        CL
  D:00FAH         PUBLIC        CCAP0H
  D:00FBH         PUBLIC        CCAP1H
  D:00EAH         PUBLIC        CCAP0L
  D:00EBH         PUBLIC        CCAP1L
  B:00A8H.4       PUBLIC        ES
  D:00B8H         PUBLIC        IP
  B:00B8H.4       PUBLIC        PS
BL51 BANKED LINKER/LOCATER V6.05                                                      07/31/2012  00:51:22  PAGE 9


  D:00D9H         PUBLIC        CMOD
  D:00D8H         PUBLIC        CCON
  C:1961H         PUBLIC        main
  D:0098H         PUBLIC        SCON
  D:0089H         PUBLIC        TMOD
  D:0088H         PUBLIC        TCON
  C:17BAH         PUBLIC        init
  D:008EH         PUBLIC        AUXR
  B:0020H.3       PUBLIC        BIT_10MS
  B:00A8H.3       PUBLIC        ET1
  D:008DH         PUBLIC        TH1
  B:0088H.0       PUBLIC        IT0
  B:00A8H.0       PUBLIC        EX0
  B:0088H.2       PUBLIC        IT1
  B:00A8H.2       PUBLIC        EX1
  D:008BH         PUBLIC        TL1
  D:00B7H         PUBLIC        IPH
  D:009CH         PUBLIC        BRT
  D:00D0H         PUBLIC        PSW
  -------         PROC          INIT
  C:17BAH         LINE#         24
  C:17BAH         LINE#         25
  C:17BAH         LINE#         29
  C:17BCH         LINE#         79
  C:17BEH         LINE#         80
  C:17C0H         LINE#         87
  C:17C2H         LINE#         88
  C:17C4H         LINE#         93
  C:17C7H         LINE#         95
  C:17CAH         LINE#         96
  C:17CDH         LINE#         100
  C:17CFH         LINE#         101
  C:17D1H         LINE#         102
  C:17D4H         LINE#         115
  C:17D7H         LINE#         116
  C:17D9H         LINE#         117
  C:17DCH         LINE#         118
  C:17DEH         LINE#         132
  C:17E1H         LINE#         133
  C:17E3H         LINE#         134
  C:17E5H         LINE#         135
  C:17E7H         LINE#         136
  C:17EAH         LINE#         137
  C:17EDH         LINE#         144
  C:17F0H         LINE#         145
  C:17F2H         LINE#         146
  C:17F4H         LINE#         147
  C:17F6H         LINE#         148
  C:17F9H         LINE#         149
  C:17FCH         LINE#         154
  -------         ENDPROC       INIT
  -------         PROC          MAIN
  C:1961H         LINE#         171
  C:1961H         LINE#         172
  C:1961H         LINE#         173
  C:1964H         LINE#         174
  C:1967H         LINE#         176
BL51 BANKED LINKER/LOCATER V6.05                                                      07/31/2012  00:51:22  PAGE 10


  C:1967H         LINE#         177
  C:1967H         LINE#         178
  C:196AH         LINE#         179
  -------         ENDPROC       MAIN
  -------         ENDMOD        MAIN

  -------         MODULE        ZIMO
  C:0000H         SYMBOL        _ICE_DUMMY_
  D:00A8H         PUBLIC        IE
  D:00B8H         PUBLIC        IP
  D:00D8H         PUBLIC        CCON
  D:0098H         PUBLIC        SCON
  D:0088H         PUBLIC        TCON
  C:003EH         PUBLIC        tab
  C:019EH         PUBLIC        love
  C:00EEH         PUBLIC        tab1
  D:00D0H         PUBLIC        PSW
  -------         ENDMOD        ZIMO

  -------         MODULE        IR_RECEIVE
  C:0000H         SYMBOL        _ICE_DUMMY_
  X:00E4H         PUBLIC        irtime
  D:00A8H         PUBLIC        IE
  D:00B8H         PUBLIC        IP
  D:00D8H         PUBLIC        CCON
  C:0026H         PUBLIC        tim1_isr
  D:0098H         PUBLIC        SCON
  D:0088H         PUBLIC        TCON
  C:172DH         PUBLIC        Ircordpro
  C:1653H         PUBLIC        ex1_isr
  X:00E5H         PUBLIC        IRcord
  X:00E7H         PUBLIC        key_code
  B:0020H.1       PUBLIC        new_code
  B:0088H.6       PUBLIC        TR1
  X:00E8H         PUBLIC        irdata
  D:00D0H         PUBLIC        PSW
  -------         PROC          TIM1_ISR
  C:0026H         LINE#         9
  C:002CH         LINE#         11
  C:0032H         LINE#         12
  -------         ENDPROC       TIM1_ISR
  -------         PROC          EX1_ISR
  -------         DO            
  X:00E1H         SYMBOL        i
  X:00E2H         SYMBOL        p
  X:00E3H         SYMBOL        z
  B:0020H.0       SYMBOL        startflag
  -------         ENDDO         
  C:1653H         LINE#         15
  C:165EH         LINE#         19
  C:1660H         LINE#         20
  C:1663H         LINE#         21
  C:1663H         LINE#         22
  C:1673H         LINE#         23
  C:1673H         LINE#         24
  C:1678H         LINE#         25
  C:167BH         LINE#         26
BL51 BANKED LINKER/LOCATER V6.05                                                      07/31/2012  00:51:22  PAGE 11


  C:167EH         LINE#         27
  C:168DH         LINE#         28
  C:1692H         LINE#         29
  C:1692H         LINE#         30
  C:1698H         LINE#         31
  C:169EH         LINE#         32
  C:169EH         LINE#         33
  C:16B0H         LINE#         34
  C:16B5H         LINE#         35
  C:16BBH         LINE#         36
  C:16BFH         LINE#         37
  C:16BFH         LINE#         38
  C:16C1H         LINE#         39
  C:16C3H         LINE#         40
  C:16C5H         LINE#         41
  C:16C5H         LINE#         42
  C:16C7H         LINE#         44
  C:16CCH         LINE#         46
  C:16CEH         LINE#         48
  C:16CEH         LINE#         49
  C:16D3H         LINE#         50
  C:16D5H         LINE#         51
  C:16D5H         LINE#         52
  -------         ENDPROC       EX1_ISR
  -------         PROC          IRCORDPRO
  -------         DO            
  D:0005H         SYMBOL        i
  D:0004H         SYMBOL        j
  D:0006H         SYMBOL        k
  D:0003H         SYMBOL        cord
  D:0007H         SYMBOL        value
  -------         ENDDO         
  C:172DH         LINE#         54
  C:172DH         LINE#         55
  C:172DH         LINE#         59
  C:172FH         LINE#         60
  C:1731H         LINE#         61
  C:1731H         LINE#         62
  C:1733H         LINE#         63
  C:1733H         LINE#         64
  C:173EH         LINE#         65
  C:1743H         LINE#         66
  C:1743H         LINE#         67
  C:1747H         LINE#         68
  C:1749H         LINE#         70
  C:1749H         LINE#         71
  C:1749H         LINE#         72
  C:1749H         LINE#         73
  C:174FH         LINE#         74
  C:174FH         LINE#         75
  C:1753H         LINE#         76
  C:1753H         LINE#         77
  C:1754H         LINE#         78
  C:1759H         LINE#         79
  C:1765H         LINE#         80
  C:1767H         LINE#         81
  C:176CH         LINE#         82
BL51 BANKED LINKER/LOCATER V6.05                                                      07/31/2012  00:51:22  PAGE 12


  C:1774H         LINE#         84
  -------         ENDPROC       IRCORDPRO
  -------         ENDMOD        IR_RECEIVE

  -------         MODULE        DS1302
  C:0000H         SYMBOL        _ICE_DUMMY_
  B:00E0H.7       PUBLIC        ACC7
  D:00B0H         PUBLIC        P3
  X:00F9H         PUBLIC        Month
  X:00FAH         PUBLIC        Cent
  X:00FBH         PUBLIC        Week
  D:00A8H         PUBLIC        IE
  B:00B0H.5       PUBLIC        T_CLK
  X:00FCH         PUBLIC        Year
  C:192EH         PUBLIC        _R1302
  D:00B8H         PUBLIC        IP
  X:00FDH         PUBLIC        Sec
  C:0006H         PUBLIC        _W1302
  X:00FEH         PUBLIC        Day
  X:00FFH         PUBLIC        Hour
  C:1775H         PUBLIC        du1302
  D:00D8H         PUBLIC        CCON
  C:1430H         PUBLIC        _Set
  B:00B0H.7       PUBLIC        T_RST
  D:0098H         PUBLIC        SCON
  D:0088H         PUBLIC        TCON
  X:0100H         PUBLIC        starts_time
  D:00E0H         PUBLIC        ACC
  B:00B0H.6       PUBLIC        T_IO
  C:1918H         PUBLIC        _RTInputByte
  C:1939H         PUBLIC        RTOutputByte
  C:183BH         PUBLIC        _Set1302
  B:00E0H.0       PUBLIC        ACC0
  D:00D0H         PUBLIC        PSW
  -------         PROC          _SET
  D:0007H         SYMBOL        sel
  X:0115H         SYMBOL        sel_1
  -------         DO            
  X:0116H         SYMBOL        address
  X:0117H         SYMBOL        time
  X:0118H         SYMBOL        max
  X:0119H         SYMBOL        min
  -------         ENDDO         
  C:1430H         LINE#         23
  C:1435H         LINE#         24
  C:1435H         LINE#         27
  C:1446H         LINE#         28
  C:1459H         LINE#         29
  C:146DH         LINE#         30
  C:1481H         LINE#         31
  C:1495H         LINE#         33
  C:14B1H         LINE#         34
  C:14C3H         LINE#         35
  C:14D8H         LINE#         36
  C:14E7H         LINE#         38
  C:14EEH         LINE#         39
  C:150AH         LINE#         40
BL51 BANKED LINKER/LOCATER V6.05                                                      07/31/2012  00:51:22  PAGE 13


  -------         ENDPROC       _SET
  -------         PROC          L?0027
  -------         ENDPROC       L?0027
  -------         PROC          _RTINPUTBYTE
  D:0007H         SYMBOL        d
  -------         DO            
  D:0007H         SYMBOL        h
  -------         ENDDO         
  C:1918H         LINE#         51
  C:1918H         LINE#         52
  C:1918H         LINE#         54
  C:1919H         LINE#         55
  C:191BH         LINE#         56
  C:191BH         LINE#         57
  C:191FH         LINE#         58
  C:1921H         LINE#         59
  C:1923H         LINE#         60
  C:1925H         LINE#         61
  C:1927H         LINE#         62
  -------         ENDPROC       _RTINPUTBYTE
  -------         PROC          RTOUTPUTBYTE
  -------         DO            
  D:0007H         SYMBOL        h
  -------         ENDDO         
  C:1939H         LINE#         72
  C:1939H         LINE#         73
  C:1939H         LINE#         75
  C:193BH         LINE#         76
  C:193BH         LINE#         77
  C:193DH         LINE#         78
  C:1941H         LINE#         79
  C:1943H         LINE#         80
  C:1945H         LINE#         81
  C:1947H         LINE#         82
  C:1948H         LINE#         83
  -------         ENDPROC       RTOUTPUTBYTE
  -------         PROC          _W1302
  D:0007H         SYMBOL        ucAddr
  D:0005H         SYMBOL        ucDa
  C:0006H         LINE#         92
  C:0006H         LINE#         93
  C:0006H         LINE#         94
  C:0006H         LINE#         95
  C:0006H         LINE#         96
  C:0006H         LINE#         97
  C:0009H         LINE#         98
  C:000EH         LINE#         99
  C:0010H         LINE#         100
  C:0012H         LINE#         101
  -------         ENDPROC       _W1302
  -------         PROC          L?0026
  -------         ENDPROC       L?0026
  -------         PROC          _R1302
  D:0007H         SYMBOL        ucAddr
  -------         DO            
  D:0007H         SYMBOL        ucData
  -------         ENDDO         
BL51 BANKED LINKER/LOCATER V6.05                                                      07/31/2012  00:51:22  PAGE 14


  C:192EH         LINE#         110
  C:192EH         LINE#         111
  C:192EH         LINE#         113
  C:192EH         LINE#         114
  C:192EH         LINE#         115
  C:192EH         LINE#         116
  C:1931H         LINE#         117
  C:1934H         LINE#         118
  C:1936H         LINE#         119
  C:1938H         LINE#         120
  C:1938H         LINE#         121
  -------         ENDPROC       _R1302
  -------         PROC          _SET1302
  D:0001H         SYMBOL        pClock
  -------         DO            
  D:0004H         SYMBOL        h
  D:0006H         SYMBOL        ucAddr
  -------         ENDDO         
  C:183BH         LINE#         132
  C:183BH         LINE#         133
  C:183BH         LINE#         135
  C:183DH         LINE#         136
  C:1844H         LINE#         137
  C:1846H         LINE#         138
  C:1846H         LINE#         139
  C:184FH         LINE#         140
  C:1856H         LINE#         141
  C:1858H         LINE#         142
  C:185AH         LINE#         143
  C:1861H         LINE#         144
  C:1868H         LINE#         145
  -------         ENDPROC       _SET1302
  -------         PROC          DU1302
  C:1775H         LINE#         149
  C:1775H         LINE#         150
  C:1775H         LINE#         151
  C:177FH         LINE#         152
  C:1789H         LINE#         153
  C:1793H         LINE#         154
  C:179DH         LINE#         155
  C:17A7H         LINE#         156
  C:17B1H         LINE#         157
  C:17B9H         LINE#         162
  -------         ENDPROC       DU1302
  -------         ENDMOD        DS1302

  -------         MODULE        SHOWTIME
  C:0000H         SYMBOL        _ICE_DUMMY_
  D:0080H         PUBLIC        P0
  D:0090H         PUBLIC        P1
  D:00A8H         PUBLIC        IE
  D:00B8H         PUBLIC        IP
  B:0020H.4       PUBLIC        flag
  D:00D8H         PUBLIC        CCON
  D:0098H         PUBLIC        SCON
  D:0088H         PUBLIC        TCON
  X:011CH         PUBLIC        id
BL51 BANKED LINKER/LOCATER V6.05                                                      07/31/2012  00:51:22  PAGE 15


  C:07DEH         PUBLIC        display
  D:00D0H         PUBLIC        PSW
  -------         PROC          DISPLAY
  -------         DO            
  X:0115H         SYMBOL        i
  -------         ENDDO         
  C:07DEH         LINE#         6
  C:07DEH         LINE#         7
  C:07DEH         LINE#         10
  C:07EDH         LINE#         11
  C:07EDH         LINE#         12
  C:080BH         LINE#         13
  C:0823H         LINE#         14
  C:0828H         LINE#         15
  C:0830H         LINE#         16
  C:0833H         LINE#         17
  C:0836H         LINE#         18
  C:083CH         LINE#         19
  C:084BH         LINE#         20
  C:084BH         LINE#         21
  C:086AH         LINE#         22
  C:0882H         LINE#         24
  C:0887H         LINE#         25
  C:088FH         LINE#         26
  C:0892H         LINE#         27
  C:0895H         LINE#         28
  C:089BH         LINE#         29
  C:08A0H         LINE#         30
  C:08A0H         LINE#         31
  C:08B4H         LINE#         32
  C:08C4H         LINE#         33
  C:08C9H         LINE#         34
  C:08CFH         LINE#         35
  C:08CFH         LINE#         38
  C:08CFH         LINE#         39
  C:08DBH         LINE#         40
  C:08DEH         LINE#         41
  C:08E1H         LINE#         45
  C:08ECH         LINE#         46
  C:08ECH         LINE#         47
  C:08F0H         LINE#         48
  C:08F0H         LINE#         49
  C:08F3H         LINE#         50
  C:08F6H         LINE#         51
  C:08FBH         LINE#         52
  C:0901H         LINE#         53
  C:0901H         LINE#         56
  C:0901H         LINE#         57
  C:090DH         LINE#         58
  C:0910H         LINE#         59
  C:0913H         LINE#         61
  C:0918H         LINE#         62
  C:0918H         LINE#         63
  C:091BH         LINE#         64
  C:091EH         LINE#         65
  C:0923H         LINE#         66
  C:092FH         LINE#         67
BL51 BANKED LINKER/LOCATER V6.05                                                      07/31/2012  00:51:22  PAGE 16


  C:0932H         LINE#         68
  C:0935H         LINE#         69
  C:093BH         LINE#         70
  C:093CH         LINE#         73
  C:093CH         LINE#         74
  C:093CH         LINE#         76
  C:093CH         LINE#         77
  C:094BH         LINE#         78
  C:094BH         LINE#         79
  C:0969H         LINE#         80
  C:0981H         LINE#         82
  C:0986H         LINE#         83
  C:098EH         LINE#         84
  C:0991H         LINE#         85
  C:0994H         LINE#         86
  C:099AH         LINE#         87
  C:09A9H         LINE#         88
  C:09A9H         LINE#         89
  C:09C8H         LINE#         90
  C:09E0H         LINE#         91
  C:09E5H         LINE#         92
  C:09EBH         LINE#         93
  C:09EBH         LINE#         96
  C:09EBH         LINE#         97
  C:09F3H         LINE#         98
  C:09F6H         LINE#         99
  C:09F9H         LINE#         102
  C:09F9H         LINE#         103
  C:09FEH         LINE#         104
  C:09FEH         LINE#         105
  C:0A12H         LINE#         106
  C:0A22H         LINE#         107
  C:0A27H         LINE#         108
  C:0A2DH         LINE#         109
  C:0A2DH         LINE#         112
  C:0A2DH         LINE#         113
  C:0A39H         LINE#         114
  C:0A3CH         LINE#         115
  C:0A3FH         LINE#         118
  C:0A4AH         LINE#         119
  C:0A4AH         LINE#         120
  C:0A4EH         LINE#         121
  C:0A4EH         LINE#         122
  C:0A51H         LINE#         123
  C:0A54H         LINE#         124
  C:0A59H         LINE#         125
  C:0A65H         LINE#         126
  C:0A68H         LINE#         127
  C:0A6BH         LINE#         128
  C:0A71H         LINE#         129
  C:0A76H         LINE#         130
  C:0A76H         LINE#         131
  C:0A79H         LINE#         132
  C:0A7CH         LINE#         133
  C:0A81H         LINE#         134
  C:0A87H         LINE#         135
  C:0A87H         LINE#         138
BL51 BANKED LINKER/LOCATER V6.05                                                      07/31/2012  00:51:22  PAGE 17


  C:0A87H         LINE#         139
  C:0A93H         LINE#         140
  C:0A93H         LINE#         141
  C:0A93H         LINE#         143
  C:0A96H         LINE#         145
  C:0A96H         LINE#         146
  C:0AA5H         LINE#         147
  C:0AA5H         LINE#         148
  C:0AC3H         LINE#         149
  C:0ADBH         LINE#         151
  C:0AE0H         LINE#         152
  C:0AE8H         LINE#         153
  C:0AEBH         LINE#         154
  C:0AEEH         LINE#         155
  C:0AF4H         LINE#         156
  C:0B03H         LINE#         157
  C:0B03H         LINE#         158
  C:0B22H         LINE#         159
  C:0B3AH         LINE#         160
  C:0B3FH         LINE#         161
  C:0B45H         LINE#         162
  C:0B45H         LINE#         165
  C:0B45H         LINE#         166
  C:0B4DH         LINE#         167
  C:0B50H         LINE#         168
  C:0B53H         LINE#         170
  C:0B53H         LINE#         172
  C:0B58H         LINE#         175
  C:0B63H         LINE#         176
  C:0B63H         LINE#         177
  C:0B69H         LINE#         178
  C:0B69H         LINE#         179
  C:0B6CH         LINE#         180
  C:0B6FH         LINE#         181
  C:0B74H         LINE#         182
  C:0B80H         LINE#         183
  C:0B83H         LINE#         184
  C:0B86H         LINE#         185
  C:0B8CH         LINE#         186
  C:0B92H         LINE#         187
  C:0B92H         LINE#         188
  C:0B95H         LINE#         189
  C:0B98H         LINE#         190
  C:0B9DH         LINE#         191
  C:0BA3H         LINE#         192
  C:0BA3H         LINE#         195
  C:0BA3H         LINE#         196
  C:0BAFH         LINE#         197
  C:0BB2H         LINE#         198
  C:0BB5H         LINE#         200
  C:0BB8H         LINE#         202
  C:0BB8H         LINE#         203
  C:0BC8H         LINE#         204
  C:0BC8H         LINE#         205
  C:0BE7H         LINE#         206
  C:0BFFH         LINE#         207
  C:0C04H         LINE#         208
BL51 BANKED LINKER/LOCATER V6.05                                                      07/31/2012  00:51:22  PAGE 18


  C:0C0AH         LINE#         209
  C:0C0AH         LINE#         212
  C:0C0AH         LINE#         213
  C:0C12H         LINE#         214
  C:0C15H         LINE#         215
  C:0C18H         LINE#         217
  C:0C28H         LINE#         218
  C:0C28H         LINE#         219
  C:0C46H         LINE#         220
  C:0C5EH         LINE#         221
  C:0C63H         LINE#         222
  C:0C69H         LINE#         223
  C:0C69H         LINE#         226
  C:0C69H         LINE#         227
  C:0C71H         LINE#         229
  C:0C71H         LINE#         230
  C:0C74H         LINE#         231
  C:0C77H         LINE#         234
  C:0C7DH         LINE#         235
  C:0C7DH         LINE#         236
  C:0C91H         LINE#         237
  C:0CA1H         LINE#         238
  C:0CA6H         LINE#         239
  C:0CACH         LINE#         240
  C:0CACH         LINE#         243
  C:0CACH         LINE#         244
  C:0CB8H         LINE#         245
  C:0CBBH         LINE#         246
  C:0CBEH         LINE#         249
  C:0CC9H         LINE#         250
  C:0CC9H         LINE#         251
  C:0CCFH         LINE#         252
  C:0CCFH         LINE#         253
  C:0CD2H         LINE#         254
  C:0CD5H         LINE#         255
  C:0CDAH         LINE#         256
  C:0CE6H         LINE#         257
  C:0CE9H         LINE#         258
  C:0CECH         LINE#         259
  C:0CF2H         LINE#         260
  C:0CF2H         LINE#         263
  C:0CF2H         LINE#         264
  C:0CF8H         LINE#         265
  C:0CF8H         LINE#         266
  C:0CFBH         LINE#         267
  C:0CFEH         LINE#         268
  C:0D03H         LINE#         269
  C:0D09H         LINE#         270
  C:0D09H         LINE#         273
  C:0D09H         LINE#         274
  C:0D15H         LINE#         275
  C:0D18H         LINE#         276
  C:0D1BH         LINE#         278
  C:0D1EH         LINE#         280
  C:0D1EH         LINE#         281
  C:0D2EH         LINE#         282
  C:0D2EH         LINE#         283
BL51 BANKED LINKER/LOCATER V6.05                                                      07/31/2012  00:51:22  PAGE 19


  C:0D4DH         LINE#         284
  C:0D65H         LINE#         286
  C:0D6AH         LINE#         287
  C:0D72H         LINE#         288
  C:0D75H         LINE#         289
  C:0D78H         LINE#         290
  C:0D88H         LINE#         291
  C:0D88H         LINE#         292
  C:0DA6H         LINE#         293
  C:0DBEH         LINE#         294
  C:0DC3H         LINE#         295
  C:0DC9H         LINE#         296
  C:0DC9H         LINE#         299
  C:0DC9H         LINE#         300
  C:0DD1H         LINE#         301
  C:0DD1H         LINE#         302
  C:0DD4H         LINE#         303
  C:0DD7H         LINE#         306
  C:0DDDH         LINE#         307
  C:0DDDH         LINE#         308
  C:0DF1H         LINE#         309
  C:0E01H         LINE#         310
  C:0E06H         LINE#         311
  C:0E0CH         LINE#         312
  C:0E0CH         LINE#         316
  C:0E0CH         LINE#         317
  C:0E0FH         LINE#         318
  C:0E12H         LINE#         319
  C:0E1EH         LINE#         322
  C:0E29H         LINE#         323
  C:0E29H         LINE#         324
  C:0E2FH         LINE#         325
  C:0E2FH         LINE#         326
  C:0E32H         LINE#         327
  C:0E35H         LINE#         328
  C:0E3AH         LINE#         329
  C:0E3DH         LINE#         330
  C:0E3DH         LINE#         333
  C:0E3DH         LINE#         334
  C:0E49H         LINE#         335
  C:0E4CH         LINE#         336
  C:0E4FH         LINE#         338
  C:0E51H         LINE#         340
  C:0E51H         LINE#         341
  C:0E61H         LINE#         342
  C:0E61H         LINE#         343
  C:0E7DH         LINE#         344
  C:0E95H         LINE#         345
  C:0E9AH         LINE#         346
  C:0E9DH         LINE#         347
  C:0E9DH         LINE#         350
  C:0E9DH         LINE#         351
  C:0EA5H         LINE#         352
  C:0EA5H         LINE#         353
  C:0EA8H         LINE#         354
  C:0EABH         LINE#         356
  -------         ENDPROC       DISPLAY
BL51 BANKED LINKER/LOCATER V6.05                                                      07/31/2012  00:51:22  PAGE 20


  -------         ENDMOD        SHOWTIME

  -------         MODULE        UART
  C:0000H         SYMBOL        _ICE_DUMMY_
  D:00A0H         PUBLIC        P2
  X:0000H         PUBLIC        ReceState
  C:1949H         PUBLIC        _Send_data
  X:0001H         PUBLIC        ReceVeryfy
  X:0002H         PUBLIC        ReceCount
  D:00A8H         PUBLIC        IE
  B:00A8H.4       PUBLIC        ES
  D:00B8H         PUBLIC        IP
  B:0098H.0       PUBLIC        RI
  B:0098H.1       PUBLIC        TI
  D:00D8H         PUBLIC        CCON
  D:0099H         PUBLIC        SBUF
  D:0098H         PUBLIC        SCON
  D:0088H         PUBLIC        TCON
  X:0003H         PUBLIC        ucControlCode
  X:0004H         PUBLIC        ucLength
  X:0005H         PUBLIC        ucDataBuff
  B:0020H.5       PUBLIC        uart_rBIT
  C:1118H         PUBLIC        MAIN_RS_INT
  D:00D0H         PUBLIC        PSW
  -------         PROC          _SEND_DATA
  D:0007H         SYMBOL        d
  C:1949H         LINE#         27
  C:1949H         LINE#         28
  C:1949H         LINE#         29
  C:194BH         LINE#         30
  C:194DH         LINE#         31
  C:1950H         LINE#         32
  C:1952H         LINE#         33
  C:1954H         LINE#         34
  -------         ENDPROC       _SEND_DATA
  -------         PROC          MAIN_RS_INT
  -------         DO            
  D:0007H         SYMBOL        DataTemp
  X:0114H         SYMBOL        i
  -------         ENDDO         
  C:1118H         LINE#         36
  C:1135H         LINE#         41
  C:113BH         LINE#         42
  C:113BH         LINE#         43
  C:113DH         LINE#         45
  C:113FH         LINE#         47
  C:1153H         LINE#         48
  C:1153H         LINE#         49
  C:1153H         LINE#         50
  C:1158H         LINE#         51
  C:1158H         LINE#         52
  C:115DH         LINE#         53
  C:115DH         LINE#         54
  C:115FH         LINE#         55
  C:115FH         LINE#         56
  C:1164H         LINE#         57
  C:116AH         LINE#         58
BL51 BANKED LINKER/LOCATER V6.05                                                      07/31/2012  00:51:22  PAGE 21


  C:1170H         LINE#         59
  C:1172H         LINE#         60
  C:1172H         LINE#         61
  C:1177H         LINE#         62
  C:117DH         LINE#         63
  C:1183H         LINE#         64
  C:1185H         LINE#         65
  C:1185H         LINE#         66
  C:1193H         LINE#         67
  C:1193H         LINE#         68
  C:1199H         LINE#         69
  C:11A5H         LINE#         70
  C:11ABH         LINE#         72
  C:11ADH         LINE#         74
  C:11ADH         LINE#         75
  C:11B4H         LINE#         76
  C:11B4H         LINE#         78
  C:11B6H         LINE#         79
  C:11B8H         LINE#         80
  C:11BEH         LINE#         82
  C:11C0H         LINE#         84
  C:11C0H         LINE#         85
  C:11C0H         LINE#         86
  C:11C0H         LINE#         87
  C:11C0H         LINE#         88
  C:11C2H         LINE#         89
  C:11C2H         LINE#         90
  C:11C6H         LINE#         91
  C:11C6H         LINE#         92
  C:11C8H         LINE#         93
  C:11C8H         LINE#         94
  C:11C8H         LINE#         95
  C:11CAH         LINE#         96
  C:11CAH         LINE#         97
  C:11CFH         LINE#         98
  C:11CFH         LINE#         99
  C:11CFH         LINE#         101
  C:11D5H         LINE#         102
  C:11D5H         LINE#         103
  C:11D7H         LINE#         104
  C:11EDH         LINE#         105
  C:11EDH         LINE#         106
  C:11EDH         LINE#         107
  C:1201H         LINE#         108
  C:1201H         LINE#         109
  C:120AH         LINE#         110
  C:1212H         LINE#         111
  C:1212H         LINE#         112
  C:1214H         LINE#         113
  C:1214H         LINE#         115
  C:1226H         LINE#         116
  C:1226H         LINE#         117
  C:1244H         LINE#         118
  C:124CH         LINE#         119
  C:125AH         LINE#         120
  C:1260H         LINE#         121
  C:1260H         LINE#         122
BL51 BANKED LINKER/LOCATER V6.05                                                      07/31/2012  00:51:22  PAGE 22


  C:1266H         LINE#         123
  C:126CH         LINE#         124
  C:1272H         LINE#         125
  C:127CH         LINE#         126
  C:1285H         LINE#         127
  C:1285H         LINE#         129
  C:128AH         LINE#         130
  C:128CH         LINE#         132
  C:128CH         LINE#         133
  C:128EH         LINE#         142
  C:1290H         LINE#         143
  C:1290H         LINE#         144
  C:1290H         LINE#         145
  C:1290H         LINE#         146
  C:1290H         LINE#         148
  C:1290H         LINE#         150
  C:1290H         LINE#         157
  -------         ENDPROC       MAIN_RS_INT
  -------         ENDMOD        UART

  -------         MODULE        EEPROM58
  C:0000H         SYMBOL        _ICE_DUMMY_
  C:18BDH         PUBLIC        _sector_erase
  D:00A8H         PUBLIC        IE
  D:00C5H         PUBLIC        IAP_CMD
  C:1897H         PUBLIC        _byte_program
  D:00B8H         PUBLIC        IP
  D:00C3H         PUBLIC        IAP_ADDRH
  D:00C4H         PUBLIC        IAP_ADDRL
  D:00D8H         PUBLIC        CCON
  X:011AH         PUBLIC        my_unTemp16
  D:0098H         PUBLIC        SCON
  C:186FH         PUBLIC        _byte_read
  D:0088H         PUBLIC        TCON
  D:00C7H         PUBLIC        IAP_CONTR
  D:00C2H         PUBLIC        IAP_DATA
  D:00C6H         PUBLIC        IAP_TRIG
  C:1955H         PUBLIC        IAP_Disable
  D:00D0H         PUBLIC        PSW
  -------         PROC          _BYTE_READ
  D:0006H         SYMBOL        add
  C:186FH         LINE#         35
  C:186FH         LINE#         36
  C:186FH         LINE#         37
  C:1872H         LINE#         38
  C:1875H         LINE#         39
  C:1878H         LINE#         41
  C:1880H         LINE#         42
  C:1886H         LINE#         43
  C:188AH         LINE#         46
  C:188DH         LINE#         47
  C:1890H         LINE#         48
  C:1891H         LINE#         50
  C:1894H         LINE#         52
  C:1896H         LINE#         53
  -------         ENDPROC       _BYTE_READ
  -------         PROC          _BYTE_PROGRAM
BL51 BANKED LINKER/LOCATER V6.05                                                      07/31/2012  00:51:22  PAGE 23


  D:0006H         SYMBOL        add
  D:0005H         SYMBOL        ch
  C:1897H         LINE#         56
  C:1897H         LINE#         57
  C:1897H         LINE#         58
  C:189AH         LINE#         59
  C:189DH         LINE#         61
  C:18A5H         LINE#         62
  C:18ABH         LINE#         63
  C:18AFH         LINE#         65
  C:18B3H         LINE#         67
  C:18B6H         LINE#         68
  C:18B9H         LINE#         69
  C:18BAH         LINE#         71
  -------         ENDPROC       _BYTE_PROGRAM
  -------         PROC          _SECTOR_ERASE
  D:0006H         SYMBOL        add
  C:18BDH         LINE#         76
  C:18BDH         LINE#         77
  C:18BDH         LINE#         78
  C:18C0H         LINE#         79
  C:18C3H         LINE#         81
  C:18CBH         LINE#         82
  C:18D1H         LINE#         83
  C:18D5H         LINE#         86
  C:18D8H         LINE#         87
  C:18DBH         LINE#         88
  C:18DCH         LINE#         90
  -------         ENDPROC       _SECTOR_ERASE
  -------         PROC          IAP_DISABLE
  C:1955H         LINE#         94
  C:1955H         LINE#         95
  C:1955H         LINE#         98
  C:1958H         LINE#         99
  C:195AH         LINE#         100
  C:195CH         LINE#         101
  C:195EH         LINE#         102
  C:1960H         LINE#         103
  -------         ENDPROC       IAP_DISABLE
  -------         ENDMOD        EEPROM58

  -------         MODULE        ?C?CLDPTR
  C:1511H         PUBLIC        ?C?CLDPTR
  -------         ENDMOD        ?C?CLDPTR

  -------         MODULE        ?C?UIDIV
  C:152AH         PUBLIC        ?C?UIDIV
  -------         ENDMOD        ?C?UIDIV

  -------         MODULE        ?C?IILDX
  C:157FH         PUBLIC        ?C?IILDX
  -------         ENDMOD        ?C?IILDX

  -------         MODULE        ?C?OFFXADD
  C:1595H         PUBLIC        ?C?OFFXADD
  -------         ENDMOD        ?C?OFFXADD

BL51 BANKED LINKER/LOCATER V6.05                                                      07/31/2012  00:51:22  PAGE 24


  -------         MODULE        ?C?CCASE
  C:15A1H         PUBLIC        ?C?CCASE
  -------         ENDMOD        ?C?CCASE

Program Size: data=25.6 xdata=285 code=6496
LINK/LOCATE RUN COMPLETE.  0 WARNING(S),  0 ERROR(S)
